:020000020000FC
:020000000BC033
:020006002CC00C
:1000160041C00FED0DBF0FEF0ABB00E00BBB03E0C5
:1000260007BB04E008BB02E000BF03E003BF0FEF1D
:1000360006BF02E009BF00E20BBF04E000BD00E31B
:1000460005BF00E808B90BE000B96627BB27CC2737
:10005600AA27FF2478948895FECF26B3209522FD03
:1000660002C0CC27C2BF22FF12C002B70330CF05A1
:1000760070F00533CF0510F01BD009C0330F441FB5
:10008600551FA39502B70D30CF0508F0339500E252
:1000960005BF1895C395C43008F4189509D066278E
:1000A600BB2700E00BBBCC27C2BF00E305BF1895FA
:1000B600A43119F407D0AA270895332744275527D2
:1000C600AA270895732FCA01082F8095709583700B
:1000D600969507959695079593700717980709F0D3
:1000E6001AC080FF08C0603029F408B300FDC0982C
:1000F60000FFC09A62E081FF08C0B03029F408B35F
:1001060001FDC19801FFC19AB2E0002706136A9566
:080116000B13BA957BBB0895A1
:00000001FF
